:020000021000EC
:04F800000C9446FC22
:020000021000EC
:14F88C0001E005BF02E005BFCFEFD0E1CDBFDEBFC051D04064
:14F8A0000AEA08830024E0E0F1E012E0E430F10711F001928E
:14F8B400FBCF0083ECE8F8EFA0E0B1E018EF01E00BBFEC3851
:14F8C800F10721F0D89531960D92F9CF0E942AFDFFCF20D001
:14F8DC00F80120936800E89508951AD0F901080131E0309329
:14F8F0006800E8950895F80120FD2093680007911691089575
:14F90400002E19E010936800E895089505D0B1E1B093680091
:14F91800E8950895B0916800B0FDFCCF0895AA92BA9275D036
:14F92C00A02E73D03A2C202E3092010120920001322C2224E7
:14F940003092030120920201ABBEB990A99008950E946EFDA3
:14F95400219700240882CC244427552715C059D0A02E57D06F
:14F96800E02E2E2C3324322C22246A2D7727620D731D2A2C9E
:14F97C00200EC20C9A018B010E9473FC4E5F5F4F4030E1E0B7
:14F990005E0738F340D0E02EC01611F0002738C023E000912B
:14F9A4000201109103010E946DFC25E000910201109103015E
:14F9B8000E946DFC0E9488FC442755271BC02227009102016B
:14F9CC0010910301040F151F0E947BFC7801B701CB01807035
:14F9E0001C01232C3324CB019070820D931D28803324280E10
:14F9F400391E28824E5F5F4F4030E1E05E0708F30880C014B6
:14FA080011F0002701C001E021960C9463FD0027112712C038
:14FA1C00A8950E5F1F4F015010408AEF9FEFA0E0B0E01801ED
:14FA30004424552482159305A405B5050CF402C05F9BECCFD8
:14FA44000CB1089501C0A8955D9BFDCF0CB9089581E083B993
:14FA580080E189B988E18AB986E880939500D7DF0EE3EEDFC1
:14FA6C00D4DF0C3311F504E5E9DF04E4E7DF00E7E5DF03E69B
:14FA8000E3DF04E3E1DFC7DF01E2DEDF13C0A8954ADF809179
:14FA94000001909101018F3FEFEF9E0709F409C055DF0023CC
:14FAA80019F001E2CDDF02C000E4CADFECCF22242BBE81E018
:14FABC0085BF25BE0C9400000895A990B990C990D990E99015
:14FAD000F990499159916991799108957A936A935A934A9360
:0EFAE400FA92EA92DA92CA92BA92AA9208951F
:00000001FF
